BL51 BANKED LINKER/LOCATER V5.03                                                        11/28/2007  10:32:21  PAGE 1


BL51 BANKED LINKER/LOCATER V5.03, INVOKED BY:
C:\KEIL\C51\BIN\BL51.EXE .\out\main.obj TO .\out\EEPROM_ASM PRINT (.\EEPROM_ASM.m51) RAMSIZE (256)


INPUT MODULES INCLUDED:
  .\out\main.obj (MAIN)


LINK MAP OF MODULE:  .\out\EEPROM_ASM (MAIN)


            TYPE    BASE      LENGTH    RELOCATION   SEGMENT NAME
            -----------------------------------------------------

            * * * * * * *   D A T A   M E M O R Y   * * * * * * *
            REG     0000H     0008H     ABSOLUTE     "REG BANK 0"

            * * * * * * *   C O D E   M E M O R Y   * * * * * * *
            CODE    0000H     01FDH     ABSOLUTE     



SYMBOL TABLE OF MODULE:  .\out\EEPROM_ASM (MAIN)

  VALUE           TYPE          NAME
  ----------------------------------

  -------         MODULE        MAIN
  D:0021H         SYMBOL        BYTE_ADDR_HIGH
  D:0022H         SYMBOL        BYTE_ADDR_LOW
  C:0112H         SYMBOL        BYTE_PROGRAM
  C:0172H         SYMBOL        BYTE_PROGRAM11
  C:018DH         SYMBOL        BYTE_PROGRAM21
  C:016AH         SYMBOL        CHANGE_DATA1
  C:0185H         SYMBOL        CHANGE_DATA2
  C:01AAH         SYMBOL        DISABLE_EXPAND_RAM
  D:0083H         SYMBOL        DPH
  D:0082H         SYMBOL        DPL
  B:00A8H.7       SYMBOL        EA
  C:01A6H         SYMBOL        ENABLE_EXPAND_RAM
  D:00F4H         SYMBOL        ISP_ADDRH
  D:00F5H         SYMBOL        ISP_ADDRL
  C:01C3H         SYMBOL        ISP_BYTE_PROGRAM
  C:01D4H         SYMBOL        ISP_BYTE_READ
  D:00F7H         SYMBOL        ISP_CMD
  D:00F6H         SYMBOL        ISP_DATA
  C:01BDH         SYMBOL        ISP_DISABLE
  C:01AEH         SYMBOL        ISP_ENABLE
  N:0080H         SYMBOL        ISP_IAP_BYTE_PROGRAM
  N:0082H         SYMBOL        ISP_IAP_SECTOR_ERASE
  C:01E3H         SYMBOL        ISP_SECTOR_ERASE
  D:0020H         SYMBOL        ONE_DATA
  D:00A0H         SYMBOL        P2
  D:00B0H         SYMBOL        P3
  C:0165H         SYMBOL        PAGE_ERASE1
  C:0108H         SYMBOL        PAGE_ERASE_2600
  D:00B5H         SYMBOL        RCON
  C:0123H         SYMBOL        READ_DATA
BL51 BANKED LINKER/LOCATER V5.03                                                      11/28/2007  10:32:21  PAGE 2


  C:012BH         SYMBOL        READ_DATA1
  C:013BH         SYMBOL        READ_DATA2
  C:0143H         SYMBOL        READ_DATA3
  D:00BFH         SYMBOL        SCONF
  D:0023H         SYMBOL        SECTOR_FIRST_BYTE_ADDR_HIGH
  D:0024H         SYMBOL        SECTOR_FIRST_BYTE_ADDR_LOW
  C:0100H         SYMBOL        START
  C:0000H         LINE#         16
  C:0100H         LINE#         39
  C:0103H         LINE#         40
  C:0106H         LINE#         41
  C:0108H         LINE#         46
  C:010BH         LINE#         47
  C:010DH         LINE#         53
  C:0110H         LINE#         54
  C:0112H         LINE#         56
  C:0115H         LINE#         57
  C:0118H         LINE#         58
  C:011AH         LINE#         59
  C:011CH         LINE#         60
  C:011DH         LINE#         61
  C:011FH         LINE#         62
  C:0120H         LINE#         63
  C:0123H         LINE#         73
  C:0126H         LINE#         74
  C:0129H         LINE#         75
  C:012BH         LINE#         77
  C:012EH         LINE#         78
  C:0131H         LINE#         79
  C:0133H         LINE#         80
  C:0134H         LINE#         81
  C:0135H         LINE#         82
  C:0136H         LINE#         83
  C:0138H         LINE#         84
  C:013BH         LINE#         93
  C:013EH         LINE#         94
  C:0141H         LINE#         95
  C:0143H         LINE#         97
  C:0146H         LINE#         98
  C:0149H         LINE#         99
  C:014BH         LINE#         100
  C:014CH         LINE#         101
  C:014DH         LINE#         102
  C:014EH         LINE#         103
  C:0150H         LINE#         104
  C:0153H         LINE#         109
  C:0155H         LINE#         110
  C:0158H         LINE#         111
  C:015AH         LINE#         112
  C:015BH         LINE#         113
  C:015CH         LINE#         118
  C:015EH         LINE#         119
  C:0161H         LINE#         120
  C:0163H         LINE#         121
  C:0164H         LINE#         122
  C:0165H         LINE#         127
  C:0168H         LINE#         128
BL51 BANKED LINKER/LOCATER V5.03                                                      11/28/2007  10:32:21  PAGE 3


  C:016AH         LINE#         136
  C:016DH         LINE#         137
  C:016FH         LINE#         138
  C:0172H         LINE#         140
  C:0173H         LINE#         141
  C:0174H         LINE#         142
  C:0177H         LINE#         143
  C:017AH         LINE#         144
  C:017CH         LINE#         145
  C:017EH         LINE#         146
  C:017FH         LINE#         147
  C:0180H         LINE#         148
  C:0182H         LINE#         149
  C:0185H         LINE#         157
  C:0188H         LINE#         158
  C:018BH         LINE#         159
  C:018DH         LINE#         161
  C:018EH         LINE#         162
  C:018FH         LINE#         163
  C:0192H         LINE#         164
  C:0195H         LINE#         165
  C:0197H         LINE#         166
  C:0199H         LINE#         167
  C:019AH         LINE#         168
  C:019BH         LINE#         169
  C:019DH         LINE#         170
  C:01A0H         LINE#         171
  C:01A2H         LINE#         172
  C:01A4H         LINE#         173
  C:01A6H         LINE#         178
  C:01A9H         LINE#         179
  C:01AAH         LINE#         184
  C:01ADH         LINE#         185
  C:01AEH         LINE#         190
  C:01B0H         LINE#         191
  C:01B3H         LINE#         192
  C:01B6H         LINE#         193
  C:01B9H         LINE#         194
  C:01BCH         LINE#         195
  C:01BDH         LINE#         200
  C:01C0H         LINE#         201
  C:01C2H         LINE#         202
  C:01C3H         LINE#         207
  C:01C5H         LINE#         208
  C:01C8H         LINE#         209
  C:01CBH         LINE#         210
  C:01CEH         LINE#         211
  C:01D1H         LINE#         212
  C:01D3H         LINE#         213
  C:01D4H         LINE#         218
  C:01D7H         LINE#         219
  C:01DAH         LINE#         220
  C:01DBH         LINE#         221
  C:01DEH         LINE#         222
  C:01E1H         LINE#         223
  C:01E2H         LINE#         224
  C:01E3H         LINE#         229
BL51 BANKED LINKER/LOCATER V5.03                                                      11/28/2007  10:32:21  PAGE 4


  C:01E5H         LINE#         230
  C:01E8H         LINE#         231
  C:01EBH         LINE#         232
  C:01EEH         LINE#         233
  C:01F1H         LINE#         234
  C:01F3H         LINE#         235
  -------         ENDMOD        MAIN

Program Size: data=8.0 xdata=0 code=509
LINK/LOCATE RUN COMPLETE.  0 WARNING(S),  0 ERROR(S)
